:020000040000FA
:0400000023EF00F0FA
:020004000000FA
:040008000FEF00F006
:040018000FEF00F0F6
:04001C001000106E52
:10002000D838116EF2B402D01CEF00F04386282EAF
:1000300003D04484640E286E1138D86E103A1038FC
:10004000F294F28E10003FEC02F0416AF29EF29AB6
:10005000F294E8EC0CF0F4EC09F0A4EC04F072EC8F
:1000600004F074EC02F09488948C93808A988B8AC4
:10007000C9EC09F0C9EC09F082A809D08B9AC9EC47
:1000800009F0C9EC09F082B802D0439001D0438056
:100090008B9A8B8EC9EC09F0C9EC09F082AC09D0BF
:1000A0008B9EC9EC09F0C9EC09F082BC02D04392E6
:1000B00001D043828B9E8A82C9EC09F0C9EC09F019
:1000C00081A009D08A92C9EC09F0C9EC09F081B08D
:1000D00002D0439401D043848A92939E938C8A8E5B
:1000E0006DEC02F081AC25D08A9E6DEC02F081BCF3
:1000F00020D08A8E6DEC02F081AC1BD08A9E6DEC14
:1001000002F081BC16D08A8E6DEC02F081AC11D069
:100110008A9E6DEC02F081BC0CD000D0000E746E93
:100120008EEC04F07350E87E736E000E746E95ECE6
:1001300004F03FEC02F093EC0CF0E4EC09F072EC0C
:100140000DF0D1EC0BF0E4EC09F072EC0DF011ECD9
:100150000CF0E4EC09F072EC0DF039EC0CF0FBEC77
:1001600002F072EC0DF0000E746E8EEC04F0735021
:10017000E8AECAD05AEC0BF0E4EC09F072EC0DF0EA
:10018000939E938C456A96EC03F08A8E6DEC02F098
:1001900081AC34D08A9E6DEC02F081BC2FD08A8E67
:1001A0006DEC02F081AC2AD08A9E6DEC02F081BC2D
:1001B00025D08A8E6DEC02F081AC20D08A9E6DEC49
:1001C00002F081BC1BD0640E3B26000E3C220F0EB9
:1001D0003C6401D006D03C6207D0A00E3B6404D042
:1001E00000D03C6A640E3B6EE4EC03F0456AD4EC4C
:1001F00009F0D4EC09F0D4EC09F0C7D7452A230E56
:100200004562C3D772EC04F0040E746E8EEC04F0F9
:1002100073503B6208D0050E746E8EEC04F0735080
:100220003C6201D00ED03BC073FF040E746E95EC9F
:1002300004F03CC073FF050E746E95EC04F0A4EC62
:1002400004F072EC0DF0939E938C456A23EC03F05E
:100250008A8E6DEC02F081AC34D08A9E6DEC02F097
:1002600081BC2FD08A8E6DEC02F081AC2AD08A9EA0
:100270006DEC02F081BC25D08A8E6DEC02F081AC71
:1002800020D08A9E6DEC02F081BC1BD00A0E1E2687
:10029000000E1F22010E1F6401D006D01F6207D07E
:1002A000F40E1E6404D000D01F6A0A0E1E6E74EC99
:1002B00003F0456AD4EC09F0D4EC09F0D4EC09F071
:1002C000C7D7452A230E4562C3D774EC02F0010E4E
:1002D000746E8EEC04F073501E6208D0020E746EC1
:1002E0008EEC04F073501F6201D00ED01EC073FF5D
:1002F000010E746E95EC04F01FC073FF020E746E55
:1003000095EC04F0A4EC04F072EC04F074EC02F050
:10031000938E938CA7EC0AF043A401D003D0080E6F
:10032000326E03D0040E326E00D043A201D003D04F
:10033000040E316E03D0020E316E00D0F28E010E2B
:10034000C26E80EC06F048C021F047C020F0050ED8
:10035000C26E80EC06F048C023F047C022F043B0E4
:1003600036D021C017F020C016F023C015F022C0EF
:1003700014F02450165E2550175AD8B003D0176ACF
:10038000166A0ED00F0E176401D006D0176206D081
:10039000A00E166403D000D0438C02D0439C00D042
:1003A0002650145E2750155AD8B003D0156A146A27
:1003B00044D00F0E156401D006D0156206D0A00EF1
:1003C000146403D000D0438A38D0439A36D021C079
:1003D00015F020C014F023C017F022C016F02450EE
:1003E000145E2550155AD8B003D0156A146A0ED081
:1003F0000F0E156401D006D0156206D0A00E14644D
:1004000003D000D0438A02D0439A00D02650165E13
:100410002750175AD8B003D0176A166A0ED00F0E9D
:10042000176401D006D0176206D0A00E166403D060
:1004300000D0438C02D0439C00D043B60CD044B4CF
:10044000FBEC02F0EBEC07F099EC02F080AC76D715
:1004500007EC04F073D74396A0EC05F008EC06F027
:1004600080AC01D007D0BDEC04F0A9EC08F021EC81
:1004700005F064D707EC04F061D73DEF02F06C0E95
:10048000D36E9B8C000E936E020E946E4F0E926E86
:100490000F015C9500018A6A8B6A898E0C0E0F0130
:1004A000506F0F019992040E0F01CA6EFF0E0F01DB
:1004B000CB6E000E0F01516F0F01509B5099000140
:1004C000010EC26E100EC16E8D0EC06E950ED56EF1
:1004D000F26AF28EF28AF28C1200C9EC09F0C9ECD1
:1004E00009F0C9EC09F01200020E746E8EEC04F0F3
:1004F00073CF57F0010E746E8EEC04F073CF56F08C
:10050000270E596E100E586EA7EC07F05DC051F023
:100510005CC050F05BC04FF05AC04EF0030E4B6E03
:10052000FF0E4A6EC8EC07F04FC01DF04EC01CF025
:10053000120019C057F018C056F0270E596E100E51
:10054000586EA7EC07F05DC051F05CC050F05BC086
:100550004FF05AC04EF01DC04BF01CC04AF0C8EC22
:1005600007F0080E336207D0030E4B6EE80E4A6E9A
:10057000C8EC07F014D0040E336207D0000E4B6EA7
:10058000640E4A6EC8EC07F00AD0020E336207D040
:10059000000E4B6E0A0E4A6EC8EC07F000D0030E38
:1005A0004F6401D006D04F6209D0FF0E4E6406D0D2
:1005B00000D0030E4F6EFF0E4E6E00D04EA004D042
:1005C0000F015089000104D000000F015099000173
:1005D0004EA204D00F01508B000104D000000F0187
:1005E000509B0001D8904F324E32D8904F324E324D
:1005F0004EC051FF12008B86D4EC09F0D4EC09F008
:10060000D4EC09F0D4EC09F0D4EC09F0010EC26E80
:1006100080EC06F048C025F047C024F0050EC26EFD
:1006200080EC06F048C027F047C026F08B96D4EC4B
:1006300009F0D4EC09F0D4EC09F0D4EC09F0D4ECD6
:1006400009F044941200010E3AEC0DF0410E11EC49
:100650000DF06E0E11EC0DF0610E11EC0DF06C0E44
:1006600011EC0DF0050E11EC0DF0670E11EC0DF014
:10067000200E11EC0DF06B0E11EC0DF0690E11EC6B
:100680000DF06D0E11EC0DF0650E11EC0DF06E0E0F
:1006900011EC0DF0650E11EC0DF0740E11EC0DF077
:1006A000400E3AEC0DF0760E11EC0DF0010E11EC4F
:1006B0000DF0670E11EC0DF06B0E11EC0DF0690EE4
:1006C00011EC0DF0740E11EC0DF0010E11EC0DF0AB
:1006D000720E11EC0DF0010E11EC0DF0730E11EC19
:1006E0000DF03A0E11EC0DF04C0E3AEC0DF01FC06F
:1006F00012F01EC013F06CEC07F02A6601D005D092
:10070000300E2A2411EC0DF005D0200E2A2411EC15
:100710000DF000D0300E2B2411EC0DF0300E2C24F7
:1007200011EC0DF0570E11EC0DF01200010E3AEC29
:100730000DF0560E11EC0DF06F0E11EC0DF06E0E6B
:1007400011EC0DF0610E11EC0DF06C0E11EC0DF0D2
:100750006B0E11EC0DF0690E11EC0DF06A0E11EC40
:100760000DF0650E11EC0DF06C0E11EC0DF07A0E23
:1007700011EC0DF0010E11EC0DF0730E11EC0DF0FB
:10078000400E3AEC0DF0760E11EC0DF0010E11EC6E
:100790000DF0670E11EC0DF06B0E11EC0DF0690E03
:1007A00011EC0DF0740E11EC0DF0010E11EC0DF0CA
:1007B000720E11EC0DF0010E11EC0DF0730E11EC38
:1007C0000DF03A0E11EC0DF04B0E3AEC0DF03CC072
:1007D00012F03BC013F06CEC07F0296601D005D095
:1007E000300E292411EC0DF005D0200E292411EC37
:1007F0000DF000D0300E2A2411EC0DF0300E2B2419
:1008000011EC0DF0300E2C2411EC0DF0120043AC65
:1008100001D030D0040E326206D016503B5C175027
:100820003C5828E332D0080E326212D00A0E4A6ECB
:10083000000E4B6E16C04EF017C04FF0506A516A52
:10084000C8EC07F04E503B5C4F503C5813E31DD0B2
:10085000640E4A6E000E4B6E16C04EF017C04FF07D
:10086000506A516AC8EC07F04E503B5C4F503C5800
:1008700001E30BD0400E3AEC0DF0140E386E050E6D
:1008800011EC0DF0382EFBD7120017C036F016C051
:1008900035F0400E3AEC0DF0376A100E386E3950D4
:1008A000355CD8B001D007D0356E050E11EC0DF0D7
:1008B000382EF5D712003606D8B0F6D700D0366AF3
:1008C0003A50355ED8B001D002D0372AF8D7375029
:1008D00011EC0DF0382E01D01200000E11EC0DF0CD
:1008E000F9D71200100E4A6E000E4B6E3BC04EF050
:1008F0003CC04FF0506A516AC8EC07F04EC039F066
:10090000050E4A6E000E4B6E39C04EF04F6A506AAB
:10091000516AC8EC07F04EC03AF012007F9E7F9CEF
:100920007F807FB091EF04F012007F9E7F9C7F84D8
:10093000F29E550E7E6EAA0E7E6E7F82F28E7FB282
:100940009FEF04F07F941200010E746E8EEC04F0A1
:1009500073CF1EF0020E746E8EEC04F073CF1FF096
:10096000040E746E8EEC04F073CF3BF0050E746EC3
:100970008EEC04F073CF3CF0120019C012F018C0D6
:1009800013F06CEC07F0000E336204D0410E3AEC29
:100990000DF004D0400E3AEC0DF000D0296606D0E0
:1009A00033B604D0200E11EC0DF004D0300E292403
:1009B00011EC0DF033A604D02E0E11EC0DF000D08A
:1009C0002A660AD033B608D033B406D0296604D0DC
:1009D000200E11EC0DF004D0300E2A2411EC0DF095
:1009E00033A404D02E0E11EC0DF000D02B660ED0E7
:1009F00033B60CD033B40AD033B208D0296606D04F
:100A00002A6604D0200E11EC0DF004D0300E2B24F9
:100A100011EC0DF033A204D02E0E11EC0DF000D02D
:100A2000300E2C2411EC0DF0570E11EC0DF0200EB1
:100A300011EC0DF0200E11EC0DF0200E11EC0DF06C
:100A4000120044B003D043B801D019D0490E3AEC9B
:100A50000DF0200E11EC0DF0200E11EC0DF0200E1B
:100A600011EC0DF03E0E11EC0DF0310E11EC0DF00D
:100A70006B0E11EC0DF0060E11EC0DF01200000ED5
:100A8000346204D04A0E3AEC0DF004D0490E3AEC30
:100A90000DF000D02D6606D034B604D0200E11EC37
:100AA0000DF004D0300E2D2411EC0DF034A604D03E
:100AB0002E0E11EC0DF000D02E660AD034B608D000
:100AC00034B406D02D6604D0200E11EC0DF004D005
:100AD000300E2E2411EC0DF034A404D02E0E11ECA7
:100AE0000DF000D02F660ED034B60CD034B40AD03E
:100AF00034B208D02D6606D02E6604D0200E11EC3C
:100B00000DF004D0300E2F2411EC0DF034A204D0DF
:100B10002E0E11EC0DF000D0300E302411EC0DF043
:100B200043A807D06B0E11EC0DF0060E11EC0DF082
:100B30001200060E11EC0DF0200E11EC0DF012005B
:100B400015C012F014C013F06CEC07F0000E3AEC74
:100B50000DF043AA13D0200E11EC0DF02D0E11EC68
:100B60000DF02D0E11EC0DF02D0E11EC0DF02D0EE3
:100B700011EC0DF0560E11EC0DF01200296606D0A6
:100B800031B604D0200E11EC0DF004D0300E292423
:100B900011EC0DF031A604D02E0E11EC0DF000D0AA
:100BA0002A660AD031B608D031B406D0296604D0FE
:100BB000200E11EC0DF004D0300E2A2411EC0DF0B3
:100BC00031A404D02E0E11EC0DF000D02B660ED007
:100BD00031B60CD031B40AD031B208D0296606D073
:100BE0002A6604D0200E11EC0DF004D0300E2B2418
:100BF00011EC0DF031A204D02E0E11EC0DF000D04E
:100C0000300E2C2411EC0DF0560E11EC0DF01200EC
:100C100017C012F016C013F06CEC07F0090E3AEC96
:100C20000DF043AC16D0200E11EC0DF02D0E11EC92
:100C30000DF02D0E11EC0DF02D0E11EC0DF02D0E12
:100C400011EC0DF0410E11EC0DF0200E11EC0DF039
:100C50001200296606D032B604D0200E11EC0DF039
:100C600004D0300E292411EC0DF032A604D02E0E43
:100C700011EC0DF000D02A660AD032B608D032B49A
:100C800006D0296604D0200E11EC0DF004D0300EF1
:100C90002A2411EC0DF032A404D02E0E11EC0DF02C
:100CA00000D02A660ED032B60CD032B40AD032B29E
:100CB00008D0296606D02A6604D0200E11EC0DF06B
:100CC00004D0300E2B2411EC0DF032A204D02E0EE5
:100CD00011EC0DF000D0300E2C2411EC0DF0020EB2
:100CE000326207D06D0E11EC0DF0410E11EC0DF0DB
:100CF0001200410E11EC0DF0200E11EC0DF012005F
:100D0000500E456E00EE60F0C280B3EC09F0C28276
:100D1000C2B288EF06F0C3CFEEFFC4CFEEFF452E80
:100D2000F6D7466A00EE61F010EE63F0EF50E7642C
:100D300001D01BD0E76209D0ED52E552EF50E764D5
:100D400001D018D0E652EE5200D0E652E652010E23
:100D5000E2622CD0010EE162E9D700D0ED6AEE6AC2
:100D6000462A080E4662DED70CD0E1CFE9FFE2CF7B
:100D7000EAFFEBD7E1CFE9FFE2CFEAFFEE52E6521E
:100D8000E4D7466A00EE61F010EE63F0EF660ED035
:100D9000ED52EE660BD0EE52EE52E652E652000EE7
:100DA000EA62F4D7FF0EE962F1D70ED0E76613D0FE
:100DB000E552E66610D0E652E652010EE262F6D740
:100DC000010EE162F3D700D0ED6AEE6A462A080E02
:100DD0004662D8D71BD0EF50E76001D00BD0E76256
:100DE000EAD7ED52E552EF50E76001D008D0E65265
:100DF000EE52E1D7E1CFE9FFE2CFEAFFDCD7E1CF66
:100E0000E9FFE2CFEAFFEE52E652D5D7476A486AD9
:100E1000496A500E466E00EE60F0EE504726EE50E6
:100E20004822D8A001D0492A46064666F6D7200EA9
:100E30004726000E4822000E4922D89049324832F7
:100E40004732D890493248324732D89049324832F6
:100E50004732D890493248324732D89049324832E6
:100E60004732D890493248324732120030D8F36EB8
:100E7000D8900BD020EE00F0330EDF26DFB6F00B5B
:100E8000DFBE0F0BDE5ED9A4F7D705360636073670
:100E90000036013602360336F32EECD703380F0B3B
:100EA0000F6E03500F0B0E6E02380F0B0D6E0250BB
:100EB0000F0B0C6E01380F0B0B6E01500F0B0A6EEF
:100EC00000380F0B096E00500F0B086E1200006AFD
:100ED000016A026A036A180C296A2A6A2B6A2C6A58
:100EE000030E125CE80ED8B4135CD8A08AEF07F0AA
:100EF000030E125CD8A08AEF07F081EF07F08AEFAB
:100F000007F0126EE80E135C136ED8A01206292AA1
:100F100070EF07F0640E135CD8B095EF07F012661F
:100F200093EF07F099EF07F01206136E2A2A8AEF63
:100F300007F00A0E135CD8A0A4EF07F02B2A136E5B
:100F400099EF07F013C02CF013C02CF012005A6A6E
:100F50005B6A5C6A5D6A58505602F3CF5AF0F4CF70
:100F60005BF059505702F3CF5CF0F4CF5DF058506E
:100F70005702F3505B26F4505C22E86A5D22595018
:100F80005602F3505B26F4505C22E86A5D221200A0
:100F9000200E526E4D6A4C6AD8904E364F365036FF
:100FA00051364C364D36D8B0E0EF07F04B504D5C23
:100FB000D8A4DDEF07F04A504C5CD8A0E7EF07F06B
:100FC0004A504C5ED8A04D064B504D5E4E80522E7E
:100FD000CCEF07F0120015C057F014C056F017C040
:100FE00059F016C058F0A7EC07F07F0E526E960E1F
:100FF000536E980E546E000E556E5A50525C5B50F4
:1010000053585C5054585D50555801E207D0080EB3
:10101000316251D0020E32624ED000D0880E5A2674
:10102000130E5B22000E5C22000E5D22100E4A6E33
:10103000270E4B6E5AC04EF05BC04FF05CC050F0B4
:101040005DC051F0C8EC07F04FC019F04EC018F069
:10105000080E31620FD0020E326203D0080E336EDA
:1010600077D0080E326203D0040E336E71D0020EB8
:10107000336E6ED0040E31620FD0020E326203D096
:10108000040E336E65D0080E326203D0020E336E4A
:101090005FD0020E336E5CD0020E326203D0020EBD
:1010A000336E56D0080E326203D0020E336E50D02B
:1010B000000E336E4DD0F40E5A26010E5B22000E48
:1010C0005C22000E5D22E80E4A6E030E4B6E5AC083
:1010D0004EF05BC04FF05CC050F05DC051F0C8EC0A
:1010E00007F04FC019F04EC018F0080E31620FD053
:1010F000020E326203D0080E336E2AD0080E32621E
:1011000003D0080E336E24D0040E336E21D0040EAB
:1011100031620FD0020E326203D0080E336E18D047
:10112000080E326203D0040E336E12D0020E336EFC
:101130000FD0020E326203D0040E336E09D0080EB7
:10114000326203D0020E336E03D0000E336E00D035
:101150001200176604D0166602D044801200449034
:101160004398100E346E080E316204D03446344673
:1011700034460BD0040E316203D03446344605D0D9
:10118000020E316202D0344600D0080E326204D022
:101190003442344234420ED0040E326203D0344220
:1011A000344208D0020E3262FDD734423442344217
:1011B000344200D015C057F014C056F0270E596EB7
:1011C000100E586EA7EC07F0800E346201D00CD0E0
:1011D000400E346201D023D0200E346201D039D0C9
:1011E000100E346267D04ED0270E4B6E100E4A6E32
:1011F0005AC04EF05BC04FF05CC050F05DC051F083
:10120000C8EC07F04EC05AF04FC05BF050C05CF025
:1012100051C05DF034423442344234424BD0030E6C
:101220004B6EE80E4A6E5AC04EF05BC04FF05CC089
:1012300050F05DC051F0C8EC07F04EC05AF04FC0FE
:101240005BF050C05CF051C05DF034423442344237
:1012500031D0000E4B6E640E4A6E5AC04EF05BC029
:101260004FF05CC050F05DC051F0C8EC07F04EC0CC
:101270005AF04FC05BF050C05CF051C05DF034429A
:10128000344218D0000E4B6E0A0E4A6E5AC04EF011
:101290005BC04FF05CC050F05DC051F0C8EC07F08F
:1012A0004EC05AF04FC05BF050C05CF051C05DF0D2
:1012B000344200D017C04BF016C04AF05AC04EF06E
:1012C0005BC04FF05CC050F05DC051F0C8EC07F05F
:1012D00050C007F04FC006F04EC005F036EC07F0E6
:1012E0000F6601D00BD00FC02DF00EC02EF00DC038
:1012F0002FF00CC030F03442438834D00E6601D059
:101300000AD00EC02DF00DC02EF00CC02FF00BC077
:1013100030F0438827D00D6601D00CD00DC02DF0E1
:101320000CC02EF00BC02FF00AC030F03442344213
:10133000439818D00C6601D00BD00CC02DF00BC018
:101340002EF00AC02FF009C030F0344243980AD082
:101350000BC02DF00AC02EF009C02FF008C030F0ED
:10136000439800D01200020E3F6E290E3E6E3E2EB4
:10137000B7EF09F03F2EB7EF09F012000C0E3F6EE9
:10138000AE0E3E6E3E2EC2EF09F03F2EC2EF09F0C8
:101390001200750E3F6EE00E3E6E3E2ECDEF09F050
:1013A0003F2ECDEF09F01200050E406E910E3F6EFC
:1013B000CF0E3E6E3E2EDAEF09F03F2EDAEF09F047
:1013C000402EDAEF09F012002E0E406EA90E3F6E8D
:1013D0002E0E3E6E3E2EEAEF09F03F2EEAEF09F0A8
:1013E000402EEAEF09F0120072EC0DF0400E57ECBF
:1013F0000DF0000E11EC0DF00A0E11EC0DF0000EC8
:1014000011EC0DF00E0E11EC0DF0110E11EC0DF0B3
:10141000110E11EC0DF00E0E11EC0DF0000E11EC92
:101420000DF0020E11EC0DF0040E11EC0DF00E0E8D
:1014300011EC0DF0110E11EC0DF01F0E11EC0DF072
:10144000100E11EC0DF00E0E11EC0DF0000E11EC63
:101450000DF0020E11EC0DF0040E11EC0DF0000E6B
:1014600011EC0DF00C0E11EC0DF0040E11EC0DF062
:10147000040E11EC0DF00E0E11EC0DF0000E11EC3F
:101480000DF0050E11EC0DF00A0E11EC0DF0000E32
:1014900011EC0DF00E0E11EC0DF0110E11EC0DF023
:1014A000110E11EC0DF00E0E11EC0DF0000E11EC02
:1014B0000DF00A0E11EC0DF0000E11EC0DF0110EF6
:1014C00011EC0DF0110E11EC0DF0110E11EC0DF0F0
:1014D000110E11EC0DF00E0E11EC0DF0000E11ECD2
:1014E0000DF0020E11EC0DF0040E11EC0DF0000EDB
:1014F00011EC0DF00E0E11EC0DF0110E11EC0DF0C3
:10150000110E11EC0DF00E0E11EC0DF0000E11ECA1
:101510000DF0020E11EC0DF0040E11EC0DF00E0E9C
:1015200011EC0DF0110E11EC0DF01F0E11EC0DF081
:10153000110E11EC0DF0110E11EC0DF0000E11EC6E
:101540000DF0000E3AEC0DF072EC0DF0120072ECA2
:101550000DF0400E57EC0DF0000E11EC0DF0000EEA
:1015600011EC0DF0000E11EC0DF0000E11EC0DF071
:10157000000E11EC0DF0000E11EC0DF0000E11EC50
:101580000DF0000E11EC0DF0100E11EC0DF0100E20
:1015900011EC0DF0100E11EC0DF0100E11EC0DF021
:1015A000100E11EC0DF0100E11EC0DF0100E11ECF0
:1015B0000DF0100E11EC0DF0180E11EC0DF0180ED0
:1015C00011EC0DF0180E11EC0DF0180E11EC0DF0E1
:1015D000180E11EC0DF0180E11EC0DF0180E11ECA8
:1015E0000DF0180E11EC0DF01C0E11EC0DF01C0E90
:1015F00011EC0DF01C0E11EC0DF01C0E11EC0DF0A9
:101600001C0E11EC0DF01C0E11EC0DF01C0E11EC6B
:101610000DF01C0E11EC0DF01E0E11EC0DF01E0E57
:1016200011EC0DF01E0E11EC0DF01E0E11EC0DF074
:101630001E0E11EC0DF01E0E11EC0DF01E0E11EC35
:101640000DF01E0E11EC0DF01F0E11EC0DF01F0E23
:1016500011EC0DF01F0E11EC0DF01F0E11EC0DF042
:101660001F0E11EC0DF01F0E11EC0DF01F0E11EC02
:101670000DF01F0E11EC0DF0000E11EC0DF0000E30
:1016800011EC0DF00E0E11EC0DF0110E11EC0DF031
:10169000110E11EC0DF00A0E11EC0DF01B0E11ECF9
:1016A0000DF0000E11EC0DF0000E3AEC0DF072ECA6
:1016B0000DF0120025C012F024C013F06CEC07F0FE
:1016C000000E3AEC0DF0410E11EC0DF04E0E11EC47
:1016D0000DF0300E11EC0DF0200E11EC0DF06F0E30
:1016E00011EC0DF0660E11EC0DF0660E11EC0DF024
:1016F000730E11EC0DF0650E11EC0DF0740E11EC83
:101700000DF03A0E11EC0DF0200E11EC0DF02B50F7
:10171000300F11EC0DF02C50300F11EC0DF06D0E60
:1017200011EC0DF0560E11EC0DF027C012F026C092
:1017300013F06CEC07F0400E3AEC0DF0410E11EC9A
:101740000DF04E0E11EC0DF0310E11EC0DF0200EDF
:1017500011EC0DF06F0E11EC0DF0660E11EC0DF0AA
:10176000660E11EC0DF0730E11EC0DF0650E11EC20
:101770000DF0740E11EC0DF03A0E11EC0DF0200E80
:1017800011EC0DF02B50300F11EC0DF02C50300FF0
:1017900011EC0DF06D0E11EC0DF0560E11EC0DF07C
:1017A0001200000E3AEC0DF0500E11EC0DF0490E47
:1017B00011EC0DF0430E11EC0DF02D0E11EC0DF0AF
:1017C000650E11EC0DF0730E11EC0DF0200E11EC06
:1017D0000DF0700E11EC0DF0610E11EC0DF06E0EAF
:1017E00011EC0DF0650E11EC0DF06C0E11EC0DF01E
:1017F0006D0E11EC0DF0010E11EC0DF0720E11ECEE
:101800000DF0030E11EC0DF0470E3AEC0DF0490E01
:1018100011EC0DF0490E11EC0DF02E0E11EC0DF047
:101820001200420E3AEC0DF0760E11EC0DF0650E42
:1018300011EC0DF0720E11EC0DF07A0E11EC0DF0B2
:10184000690E11EC0DF0050E11EC0DF03A0E11ECD5
:101850000DF0020E300F11EC0DF02E0E11EC0DF00C
:10186000010E300F11EC0DF0000E300F11EC0DF0E9
:101870001200010E3AEC0DF0700E11EC0DF0610E3D
:1018800011EC0DF02D0E11EC0DF0650E11EC0DF0BC
:101890006C0E11EC0DF0650E11EC0DF06B0E11ECF1
:1018A0000DF0740E11EC0DF0720E11EC0DF06F0EC8
:1018B00011EC0DF06E0E11EC0DF0690E11EC0DF047
:1018C0006B0E11EC0DF0610E11EC0DF0430E3AECC5
:1018D0000DF0020E300F11EC0DF0000E300F11EC78
:1018E0000DF0010E300F11EC0DF0010E300F11EC68
:1018F0000DF02E0E11EC0DF0000E300F11EC0DF06E
:10190000050E300F11EC0DF02E0E11EC0DF0010E46
:10191000300F11EC0DF0050E300F11EC0DF02E0E06
:1019200011EC0DF01200410E11EC0DF0640E11ECF3
:101930000DF06A0E11EC0DF06F0E11EC0DF06E0E45
:1019400011EC0DF0200E11EC0DF0610E11EC0DF00C
:101950007A0E11EC0DF0200E11EC0DF0490E11EC89
:101960000DF0730E11EC0DF0740E11EC0DF0650E10
:1019700011EC0DF06E0E11EC0DF02C0E11EC0DF0C3
:10198000420E3AEC0DF0730E11EC0DF07A0E11ECE4
:101990000DF0650E11EC0DF0620E11EC0DF0620E03
:1019A00011EC0DF0200E11EC0DF06A0E11EC0DF0A3
:1019B000000E11EC0DF0760E11EC0DF0030E11EC93
:1019C0000DF0740E11EC0DF0210E11EC0DF0120063
:1019D000D4EC09F0D4EC09F0D4EC09F0D4EC09F023
:1019E000D4EC09F08A9A8A988B988B9A8B9C8B9E60
:1019F0008A808A828A948A96C9EC09F08A88C9EC1E
:101A000009F08A988B988B9A8B8C8B8E8A808A822D
:101A10008A948A96C9EC09F08A88C9EC09F08A98F8
:101A20001200F2AE01D002D0449201D04482F29E64
:101A30008A988A8A8A968A948A928A908B9E8B9CAC
:101A40008B9A8B98E8B08A86E8B28A84E8B48A8256
:101A5000E8B68A80E8B88B8EE8BA8B8CE8BC8B8AB3
:101A6000E8BE8B888A88B3EC09F08A9844A21200F9
:101A7000F28E12008A988A9A8A968A948A928A901A
:101A80008B9E8B9C8B9A8B88E8B08A86E8B28A847E
:101A9000E8B48A82E8B68A80E8B88B8EE8BA8B8C84
:101AA000E8BC8B8A8A88B3EC09F08A9812008A987D
:101AB0008A9A8A968A948A928A908B9E8B9C8B8A29
:101AC0008B98E8B08A86E8B28A84E8B48A82E8B65D
:101AD0008A80E8B88B8EE8BA8B8C8A88B3EC09F0E0
:101AE0008A9812008A988A9A8A868A948A928A9018
:101AF0008B9E8B9C8B9A8B988A88B3EC09F08A9882
:101B0000BEEC09F0BEEC09F01200000E3AEC0DF04C
:101B1000200E11EC0DF011EC0DF011EC0DF011ECAC
:101B20000DF011EC0DF011EC0DF011EC0DF011ECCD
:101B30000DF011EC0DF011EC0DF011EC0DF011ECBD
:101B40000DF011EC0DF011EC0DF011EC0DF011ECAD
:101B50000DF01200400E3AEC0DF0200E11EC0DF0DD
:101B600011EC0DF011EC0DF011EC0DF011EC0DF08D
:101B700011EC0DF011EC0DF011EC0DF011EC0DF07D
:101B800011EC0DF011EC0DF011EC0DF011EC0DF06D
:101B900011EC0DF011EC0DF011EC0DF01200CFEF87
:021BA0000DF046
:020000040030CA
:010000001DE2
:0100010018E6
:010002007984
:010003003CC0
:0100050009F1
:010006009168
:010008000CEB
:010009008076
:01000A000FE6
:01000B00E014
:01000C000FE4
:01000D0040B2
:0200000400F00A
:0600000000F40100A00F56
:00000001FF
